:020000040000FA
:040000006D303A28FD
:08000800A000030EA100831209
:100010008B1C32288B1031181428B11C3228643004
:10002000010203183128182800001628172818285C
:1000300019281A281B281C281D281E281F283110A3
:10004000B114A810031005190314AA0DA90DA80DC9
:10005000B00B322831152A08AF002908AE00280855
:10006000AD00B11081010B11210E8300A00E200EF6
:02007000090085
:0C007400203084008001840A6030040207
:10008000031C3C281230B000AF2183160C308505CC
:1000900087018312850187010730990000309A009B
:1000A000103083168E008312603083168F00831207
:1000B0000030831691008312C830831681008312AA
:1000C00031309000003083168C00831210308B008A
:1000D000831600309B001C141A088312BC00851D77
:1000E000F321831610309B001C141A088312BD00E4
:1000F000EB2181018E018F010B118B100B108C01F4
:100100008B1790203119A620B30B8E280310851968
:100110000314B90DF030390203192821182281285F
:100120006400311808000B1D08000B11B1103114C8
:100130001230B000051DA12832148316011383125A
:1001400008003210831601178312080031110130A4
:10015000B7008B132030370783169B001C141A0836
:100160008312A400A500C030A506103037078316FF
:100170009B001C141A088312A30000303707831653
:100180009B001C141A088312A2008B17321CCE2865
:1001900022090339A200A309A409A50922082D02F6
:1001A000031D222923082E02031D222924082F02C1
:1001B000031D222901303702031DE3283D18E328DF
:1001C0003D143E14BA2102303702031DEC28BD183D
:1001D000EC28BD143E14BC2103303702031DF52862
:1001E0003D19F5283D153E14BE2104303702031D8C
:1001F000FE28BD19FE28BD153E14C021053037026A
:10020000031D07293D1A07293D163E14C221063059
:100210003702031D1029BD1A1029BD163E14C42132
:1002200007303702031D19293D1B19293D173E14BC
:10023000C62108303702031D2229BD1B2229BD1704
:100240003E14C821B70A0930370203180800A9284C
:100250000130B600B300B400B500B70085018701D6
:10026000B1139020B30B6029031085190314B90D45
:10027000F030390203198729B40B602901303702A5
:100280000319D321023037020319D6210330370274
:100290000319D921043037020319DC210530370254
:1002A0000319DF21063037020319E2210730370234
:1002B0000319E521083037020319E8219630B4000C
:1002C000311D31293111321C6A292D090339AD0044
:1002D000AE09AF092F1CB1132F1C3129B11B3129D5
:1002E0002E183129B1178B1320303707BB002F0888
:1002F000BA009A2110303707BB002E08BA009A21A5
:1003000000303707BB002D08BA009A218B178501F2
:100310008701B70AB60109303702031C3129EB21E6
:1003200008003E1C08003E101030BB003D08BA001B
:100330009A2108008B133A0883161C159A00831221
:100340003B0883169B0055309D00AA309D009C14ED
:1003500064009C18A8291C1183128B170800FF3019
:10036000D000D415D515D615D715D915DA15DB1546
:10037000DC150800F130CB29F230CB29F430CB2941
:10038000F830CB291F30CF292F30CF294F30CF293C
:100390008F30CF290800BD050F30D2040800BD05FD
:1003A000F030D204080010308506080020308506A1
:1003B0000800213085060800223085060800183024
:1003C00087060800213087060800093087060800E4
:1003D0002930870608003D08D200031D08001130AF
:1003E000BD00D2000800B601B301B4013C1CFB29DA
:1003F000BC01BC14FD29BC013C143C08B6006400DF
:10040000012A022A032A042A052AB41B0516B41F4E
:100410000512B30BFF29B40BFF290310B60CB60865
:10042000031DFF290030BB003C08BA009A210800D8
:100430008F08031908008F01D00F322BD00A0E301D
:100440005205031D322A541D282AD4015416402A6D
:10045000D41D2D2AD4015416402A541E402AD401FA
:10046000D414402AD41C372AD4015415402A541DD0
:100470003C2AD401D415402A541E402AD4015415D4
:1004800001305205031D532A551D492AD501551621
:10049000612AD51D4E2AD5015516612A551E612A9D
:1004A000D501D514612AD51C582AD5015515612AC4
:1004B000551D5D2AD501D515612A551E612AD50124
:1004C00055150B305205031D742A561D6A2AD60194
:1004D0005616822AD61D6F2AD6015616822A561E15
:1004E000822AD601D614822AD61C792AD60156151C
:1004F000822A561D7E2AD601D615822A561E822AA7
:10050000D601561507305205031D952A571D8B2A13
:10051000D7015716A32AD71D902AD7015716A32A09
:10052000571EA32AD701D714A32AD71C9A2AD7016A
:100530005715A32A571D9F2AD701D715A32A571E3F
:10054000A32AD70157151030BC1811305205031DCE
:10055000B82A591DAE2AD9015916C62AD91DB32A5F
:10056000D9015916C62A591EC62AD901D914C62A34
:10057000D91CBD2AD9015915C62A591DC22AD9012B
:10058000D915C62A591EC62AD90159155030BC188A
:1005900051305205031DDB2A5A1DD12ADA015A16A1
:1005A000E92ADA1DD62ADA015A16E92A5A1EE92A58
:1005B000DA01DA14E92ADA1CE02ADA015A15E92A02
:1005C0005A1DE52ADA01DA15E92A5A1EE92ADA0162
:1005D0005A15E030BC18E1305205031DFE2A5B1DA0
:1005E000F42ADB015B160C2BDB1DF92ADB015B1601
:1005F0000C2B5B1E0C2BDB01DB140C2BDB1C032BED
:10060000DB015B150C2B5B1D082BDB01DB150C2BB9
:100610005B1E0C2BDB015B152030BC182130520512
:10062000031D212B5C1D172BDC015C162F2BDC1D01
:100630001C2BDC015C162F2B5C1E2F2BDC01DC1429
:100640002F2BDC1C262BDC015C152F2B5C1D2B2B90
:10065000DC01DC152F2B5C1E2F2BDC015C1591219E
:100660003D08D2005008D1000C305405031D05127E
:100670000C305505031D85120C305605031D051061
:100680000C305705031D85100C305905031D07104C
:100690000C305A05031D87120C305B05031D071231
:1006A0000C305C05031D871151080E0203187C2BCA
:1006B00012305405031D051612305505031D85160D
:1006C00012305605031D051412305705031D8514FD
:1006D00012305905031D071412305A05031D8716E1
:1006E00012305B05031D071612305C05031D8715CC
:1006F000FF305002031908008F08031D08009020E6
:1007000051080E02031C7C2B18305405031D0512E2
:1007100006305405031D051618305505031D8512B6
:1007200006305505031D851618305605031D0510A6
:1007300006305605031D051418305705031D851096
:1007400006305705031D851418305905031D071081
:1007500006305905031D071418305A05031D87126A
:1007600006305A05031D871618305B05031D071256
:1007700006305B05031D071618305C05031D871145
:0A07800006305C05031D8715080014
:084000000400030002000600A9
:02400E00CC33B1
:10420000010003000300030003000200020002009B
:1042100002000000000000000000FF00FF00FF009F
:10422000000000000000000000000000000000008E
:104230000000C000C000C000C000FF00FF00FF0081
:104240000100C300F300CF00FF00C300F300CF0064
:10425000FF00C300F300CF00FF00FF00FF00FF00DE
:10426000FF00FF00FF00FF00FF00FF00FF00FF0056
:10427000FF00FF00FF00FF00FF00FF00FF00FF0046
:10428000FF00FF00FF00FF00FF00FF00FF00FF0036
:10429000FF00FF00FF00FF00FF00FF00FF00FF0026
:1042A000FF00FF00FF00FF00FF00FF00FF00FF0016
:1042B000FF00FF00FF00FF00FF00FF00FF00FF0006
:1042C000FF00FF00FF00FF00FF00FF00FF00FF00F6
:1042D000FF00FF00FF00FF00FF00FF00FF00FF00E6
:1042E000FF00FF00FF00FF00FF00FF00FF00FF00D6
:1042F000FF00FF00FF00FF00FF00FF00FF00AA001B
:00000001FF
